:100000000C942A000C9447000C9447000C94470071
:100010000C94B3100C9447000C9447000C944700C8
:100020000C9447000C9447000C9447000C94470034
:100030000C9447000C94070B0C9447000C94470059
:100040000C9447000C9447000C9447000C94470014
:100050000C94470011241FBECFE5D8E0DEBFCDBF12
:1000600015E0A0E6B0E0E0EDF4E302C005900D92EB
:10007000A839B107D9F717E0A8E9B5E001C01D928A
:10008000AC3CB107E1F70E94D8100C94661A0C94AE
:1000900000002FE02093E6059093E7058093E805A4
:1000A0001092E90584E060E00E94C5098091FC059A
:1000B00008950F931F9388E294E00E944900182F3F
:1000C00000E089E294E00E944900080F111DC80178
:1000D0001F910F9108950F931F9386E294E00E9461
:1000E0004900182F00E087E294E00E944900080FC1
:1000F000111DC8011F910F9108950F931F9384E262
:1001000094E00E944900182F00E085E294E00E94EC
:100110004900080F111DC8011F910F9108950F93F9
:100120001F9382E294E00E944900182F00E083E2CE
:1001300094E00E944900080F111DC8011F910F9102
:1001400008950F931F9380E294E00E944900182FB6
:1001500000E081E294E00E944900080F111DC801EF
:100160001F910F91089583E094E00E944900089543
:1001700083E094E00E944900873121F481E080937C
:10018000980502C01092980580919805089520EF77
:100190002093E6059093E7058093E8056093E905D1
:1001A00084E060E00E94C50908951F93182F692F0D
:1001B00088E294E00E94C70089E294E0612F0E94E7
:1001C000C7001F9108954F925F927F928F929F92E6
:1001D000AF92BF92CF92DF92EF92FF920F931F9355
:1001E000CF93DF93082F0E946B009C01009711F4BE
:1001F0007724AEC0702E80E1801710F440E1742E99
:10020000872D90E02817390708F4722E0E945900B4
:100210004C01EC01DF70C12C90E6D92ECC0EDD1E16
:1002200080E690E00E94D60AC4010E94690B83E731
:1002300090E00E94D60ACE010E94690B8CE790E004
:100240000E94D60AC6010E94690B8AE00E94C90A70
:10025000A72CBB24C5018C0F9D1F8150904118F421
:10026000C0E0D0E037C0E12C80E1F82EEC1AFD0AA6
:1002700025014E185F0800E009C0CE018C0D9D1DC0
:100280000E944900CD53DA4F88830F5FC02FD0E022
:10029000CE15DF0590F3DD240CC08C010E0D1F1D63
:1002A0008050904A0E9449000D531A4FF8018083F4
:1002B000D3948D2D90E08415950578F30DC0C6017B
:1002C0000E944900FE01ED53FA4F80832196089465
:1002D000C11CD11CC71598F3C501880D991D0E943A
:1002E000D50081E094E060E40E94C7000E94A10074
:1002F0000E94690B89E00E94C90A8CE70E94C90A22
:100300000E948F000E94690B89E00E94C90A8CE755
:100310000E94C90A0E947D000E94690B89E00E9428
:10032000C90A8CE70E94C90A0E946B000E94690BEF
:1003300089E00E94C90A8CE70E94C90A0E945900FC
:100340000E94690B89E00E94C90A8CE70E94C90AD1
:10035000872DDF91CF911F910F91FF90EF90DF904C
:10036000CF90BF90AF909F908F907F905F904F9075
:1003700008951F93182F692F84E294E00E94C7000C
:1003800085E294E0612F0E94C7001F9108958F922B
:100390009F92AF92BF92CF92DF92EF92FF920F9314
:1003A0001F93CF93DF93182F0E94A100EC010097B9
:1003B00011F400E060C00E947D004C019C013F7080
:1003C000E12C50E4F52EE20EF31E012F113108F05E
:1003D00000E1802F90E0C817D90708F40C2FC02E39
:1003E000DD24C601820F931F8150904118F4C0E0B4
:1003F000D0E035C0C0E0D0E1C21BD30B5601AC1A2F
:10040000BD0A10E009C0FC01ED52FA4F60818E0D6B
:100410009F1D0E94C7001F5F812F90E08C179D07D2
:1004200090F310E00BC0FC01EC0FFD1FED52FA4FF2
:1004300060818050904A0E94C7001F5F812F90E02A
:100440008A159B0580F30DC0FE01ED52FA4F6081C5
:10045000C7010E94C70021960894E11CF11CC01737
:1004600098F3C601880D991D0E94B90181E094E0BE
:1004700060E20E94C700802FDF91CF911F910F9102
:10048000FF90EF90DF90CF90BF90AF909F908F90B4
:1004900008951F9389E090E06AEF0E94C7008AE008
:1004A00090E067EC0E94C7008BE090E06FE00E9454
:1004B000C7008CE090E06DEA0E94C7008DE090E0FC
:1004C00062E20E94C7008EE090E061E00E94C700F7
:1004D0008FE090E060EC0E94C70080E190E068EA65
:1004E0000E94C70081E190E060E00E94C70082E1C5
:1004F00090E062E00E94C70085E090E06FEF0E940C
:10050000C70086E090E06FEF0E94C70087E090E0B0
:100510006FEF0E94C70088E090E060E00E94C70093
:1005200081E090E060EC0E94C70082E090E061E230
:100530000E94C70083E090E060E60E94C70084E06C
:1005400090E061E00E94C7008AE190E06AE00E94CA
:10055000C7008BE190E06AE00E94C70080E094E071
:1005600061E00E94C70084E094E063E10E94C7005C
:1005700085E094E068E80E94C7008CE890E00E9463
:10058000D60A81E094E061E00E94C70083E094E035
:100590000E944900182F8EEA90E00E94D60A812F0F
:1005A0000E947D0B8AE00E94C90A133179F782EC20
:1005B00090E00E94D60A81E094E062E00E94C700C9
:1005C00083E094E00E944900182F8EEA90E00E9498
:1005D000D60A812F0E947D0B8AE00E94C90A14313D
:1005E00079F784E11F910895EF92FF920F931F9383
:1005F000939885E40E94BE09939A85E88A95F1F75D
:10060000939880E00E94BE09E82EFF2400E010E0ED
:10061000102F0F2DFE2CEE2480E00E94BE0990E0EA
:10062000A0E0B0E0E82AF92A0A2B1B2B102F0F2D8F
:10063000FE2CEE2480E00E94BE09939A282F30E021
:1006400040E050E02E293F29402B512BB901CA012F
:100650001F910F91FF90EF900895939881E00E9471
:10066000BE09939A939881E00E94BE09939A0895D7
:100670001F93182F939881E00E94BE09939A939834
:10068000112311F082E001C083E00E94BE09939A19
:100690001F9108951F939798979A939884E40E94C6
:1006A000BE09939A15E8812F8A95F1F7939880E017
:1006B0000E94BE09939A812F8A95F1F7939887E05B
:1006C0000E94BE09939A812F8A95F1F7939883E04F
:1006D0000E94BE09939A812F8A95F1F7939880E042
:1006E0000E94BE09939A812F8A95F1F7939884E02E
:1006F0000E94BE09939A812F8A95F1F7939882E51B
:100700000E94BE09939A812F8A95F1F7939883E00E
:100710000E94BE09939A812F8A95F1F7939881E3FD
:100720000E94BE09939A812F8A95F1F7939882E0EF
:100730000E94BE09939A812F8A95F1F793988EE8CB
:100740000E94BE09939A812F8A95F1F7939881E0D0
:100750000E94BE09939A812F8A95F1F7939883E0BE
:100760000E94BE09939A812F8A95F1F7939884E4A9
:100770000E94BE09939A812F8A95F1F7939880E0A1
:100780000E94BE09939A1A95F1F71F91089584B7B4
:100790008093E30514BE8898899A87B38C6087BBE1
:1007A000D798A798D6988AB38F638ABB84B38F678C
:1007B00084BBBC9A81B3886381BBC49A82B38863CB
:1007C00082BBBD9ABF9ABE98C59AC79A8E988F9AD7
:1007D0008A9808952FB78D5FF894A89591B5986180
:1007E00091BD81BD2FBF08950F931F93CF93DF93CA
:1007F000482FC0E0D0E0082F10E00F5F1F4FC80166
:100800008C0F9D1F64E570E00E94FA19382FE82FC5
:10081000E695E695E695F0E0E95AF94F808190E09B
:10082000232F277002C0959587952A95E2F780FDC2
:1008300005C02196C435D10511F7342F832FDF91E0
:10084000CF911F910F910895582F482F4F5F682F18
:100850006F5B342F3F73E32FE695E695E695F0E066
:10086000ED59F84F808190E0232F277002C09595B5
:1008700087952A95E2F780FD04C04F5F461749F738
:10088000352F832F089581E08093C10520E030E06B
:10089000F901E95AF94FD901A55BB94F90818C91C3
:1008A000981719F01092C10505C02F5F3F4F2B30EC
:1008B000310571F781E08093BD0520E030E0F9015A
:1008C000ED59F84FD901AC53B84F90818C919817DE
:1008D00019F01092BD0508952F5F3F4F2830310564
:1008E00071F7089586EE90E00E94D60A08958EE290
:1008F00091E00E94D60A80910906853010F190910E
:100900000C06892F81548830E0F4892F0E94C90A8F
:1009100080E591E00E94D60A80910E060E947D0B30
:100920008AE00E94C90AE0910C06F0E0E154F04030
:10093000DF01AD59B84F80910E068C93EC53F84F00
:100940002BC083E08093090690910B06892F815478
:10095000883020F5892F0E94C90A80910C068033C7
:1009600061F085E591E00E94D60AE0910B06F0E087
:10097000EE5DF84F8FEF80830AC08FE591E00E9413
:10098000D60AE0910B06F0E0EE5DF84F1082E091A0
:100990000B06F0E0ED57F84F1082089589E691E0DC
:1009A0000E94D60A8CE791E00E94D60A809109063F
:1009B00063E00E94870B84E991E00E94D60A80914F
:1009C0000C060E94C90A8BEA91E00E94D60A809127
:1009D0000E060E947D0B8AE00E94C90A089586B126
:1009E000866086B93098359A80B78F7180BF379A04
:1009F0003E983F983D9A87B1866087B9369A0895A8
:100A00000E94F40208950E94F4020E946C172FEFD6
:100A10003FEF4FE75BE40E94AE1520E030E040E09E
:100A20005FE30E94B41420E030E048EC50E40E9400
:100A3000B41408950E94F402643D27E7720726E685
:100A4000820720E0920708F449C0643923E972075D
:100A500029E7820720E0920728F1643721E2720734
:100A600023E8820720E0920798F0643628EE7207A8
:100A700027E8820720E0920708F411C160352FEAC9
:100A800072072CE8820720E0920708F415C121C103
:100A900064382AE572072EE7820720E0920708F003
:100AA000F1C0E3C0643B25E0720720E7820720E045
:100AB000920750F0643A2CEC720724E7820720E09A
:100AC000920708F0C5C052C0643C2EE372072BE6C3
:100AD000820720E0920708F0AEC0A0C064312CE588
:100AE000720723E5820720E09207E0F0643F29EED9
:100AF00072072CE5820720E0920750F0643E20EB5D
:100B0000720721E6820720E0920708F07AC06CC0E5
:100B1000643023E2720728E5820720E0920708F09C
:100B200056C048C064332EEC720729E4820720E0E7
:100B3000920748F0643225E972072EE4820720E02C
:100B4000920758F5E6C0643427E0720725E482076F
:100B500020E0920708F0D0C0653520E4720720E459
:100B6000820720E0920708F0BAC0B3C00E946C1759
:100B700024E130EB4AE956E40E94AE152FE833E653
:100B800045E853E40E945614E62F692F2E2F372F85
:100B9000482F562FB901CA0108950E946C172AEBFD
:100BA0003CED4FE956E40E94AE1526E43CE140E8F6
:100BB00053E4E8CF0E946C172DE73FE14FE956E47C
:100BC0000E94AE152FE03CEB40E853E4DBCF0E94DF
:100BD0006C1721E432E64EE956E40E94AE152BEA8A
:100BE00036E641E853E4CECF0E946C1725E035EAA3
:100BF0004DE956E40E94AE1523E43CE142E853E49B
:100C0000C1CF0E946C1729EC37EE4CE956E40E94E4
:100C1000AE152EEF3CED42E853E4B4CF0E946C17C2
:100C20002DE83AE24CE956E40E94AE1520E039EA9C
:100C300043E853E4A7CF0E946C1720E53DE64BE95B
:100C400056E40E94AE1529E730E844E853E49ACF11
:100C50000E946C1728ED32EF49E956E40E94AE1568
:100C60002BE632E546E853E48DCF0E946C172CE961
:100C700035E349E956E40E94AE152FE33DE447E829
:100C800053E480CF0E946C1720E638E748E956E429
:100C90000E94AE1523E334E548E853E473CF0E9485
:100CA0006C1723E23BEB47E956E40E94AE1523E7BD
:100CB00037E649E853E466CF0E946C1727EE3DEF14
:100CC00046E956E40E94AE1522E337E84AE853E4C9
:100CD00059CFAA9AE3EC75EF88E460EC57CF0E94F5
:100CE0006C1725E739E342EA56E40E94AE1528EA7C
:100CF00035EC4CE753E446CF0E946C1729E134E60B
:100D000041EA56E40E94AE1526E436EE4DE753E480
:100D100039CF0E946C172FEF3BE940EA56E40E945E
:100D2000AE1529E23BE04FE753E42CCF0E94F402DA
:100D30009B01AC01DC01CB0183539343A542B0403E
:100D40008D5C9C4CA24DB040C8F4CA01B9010E9410
:100D50006C1729ED30EA4AE457E40E94AE1522E50B
:100D600039E04CE752E40E94561442E025E00E942C
:100D7000550B82EC91E00E94E00A089586EC91E028
:100D80000E94E00AAA9A0895883248F4282F30E099
:100D9000843210F02F5F3F4F922F990F1FC0803584
:100DA00060F48852282F30E0843210F02F5F3F4FDC
:100DB000220F331F922F9F5F11C0843560F480553E
:100DC000813039F0813018F0843028F406C098E47E
:100DD00005C099E403C090E001C098E585B39F7712
:100DE0008078982B95BB0895282F82958F7082303C
:100DF00041F0833041F0882311F490E105C090E088
:100E000003C090E301C090E28BB32F70922B807CE3
:100E1000982B9BBB08950F931F93182F062F803597
:100E200008F568E20E94DA1996959695963028F4AE
:100E3000943070F4923040F009C0983069F09830E6
:100E400048F0993069F40AC081E40DC082E40BC017
:100E500083E409C084E407C085E405C086E403C0D8
:100E60008FE301C088E40E94C90A812F68E20E94D2
:100E7000DA199452943010F4137001C01770812F56
:100E80008F5F61E00E94870B8AE30E94C90A802F6E
:100E900090E024E0880F991F2A95E1F764E00E9412
:100EA000730B1F910F9108951F93CF93DF938FECD6
:100EB00091E00E94D60AC0E0D0E01C2FCE018770DE
:100EC0009070892B19F48AE00E94C90AFE01E0594A
:100ED000F84F812F60810E940B078BEE91E00E94FA
:100EE000D60A2196C435D10541F78AE00E94C90A85
:100EF000DF91CF911F910895CF92DF92EF92FF92F1
:100F00001F93182F6A017B018FEE91E00E94D60A91
:100F1000812F8695869586958F5B0E94C90A1770EA
:100F2000812F8F5F61E00E94870B8AE30E94C90ACC
:100F3000C701B6010E946C1720E030E048EC50E495
:100F40000E94B41420E030E040E053E30E94B41467
:100F500043E026E00E94550B1F91FF90EF90DF9039
:100F6000CF900895CF92DF92EF92FF920F931F934D
:100F7000CF93DF9382EF91E00E94D60A43E6E42EFE
:100F800046E0F42EC0E0D0E01C2F37E0C32ED12C79
:100F9000CC22DD22C114D10419F48AE00E94C90ACE
:100FA0008FEE91E00E94D60A012F069506950695D0
:100FB000802F8F5B0E94C90A1770812F8F5F61E0BD
:100FC0000E94870B8AE30E94C90A10E00D59184F4E
:100FD000F801808190E002C095958795CA94E2F768
:100FE00080FF1AC0F70160817181828193810E9424
:100FF0006C172DEC3CEC4CEC50E40E94B41420E057
:1010000030E040E053E30E94B41443E026E00E9445
:10101000550B8CE192E002C08EE192E00E94D60A6C
:10102000219684E090E0E80EF91EC034D10509F065
:10103000ABCFDF91CF911F910F91FF90EF90DF9099
:10104000CF9008950E9454070E94B2070895CF934D
:10105000DF9388E292E00E94D60AC7E5D6E0899144
:101060000E94780B80E20E94C90A86E0C236D80747
:10107000B1F78AE00E94C90ACBE4D6E089910E94C8
:10108000780B80E20E94C90A86E0C635D807B1F71E
:101090008AE00E94C90A85E392E00E94D60AC3E66C
:1010A000D7E089910E94780B80E20E94C90A87E00C
:1010B000CB36D807B1F78AE00E94C90AC4ECD7E062
:1010C00089910E94780B80E20E94C90A87E0CC3C9B
:1010D000D807B1F78AE00E94C90A85E492E00E942D
:1010E000D60A6091B3057091B4058091B5059091D1
:1010F000B6050E946C1720E030E04AE754E40E94F5
:10110000AE1541E027E00E94550B8BE492E00E946F
:10111000D60A82E592E00E94D60A8091C105882312
:1011200019F085E692E002C08CE692E00E94D60AB1
:1011300083E792E00E94D60A8091BD05882319F0CA
:1011400085E692E002C08CE692E00E94D60A89E829
:1011500092E00E94D60A8091BF0562E00E94870B50
:101160008AE00E94C90A8EE992E00E94D60A809124
:10117000B80562E00E94870B8AE00E94C90ADF91ED
:10118000CF91089508959CB180919905882321F409
:10119000913011F49093990580919905882361F01D
:1011A00080910906E82FF0E0E65FF94F9091620622
:1011B00090838F5F8093090608951092290686EB2D
:1011C00092E00E94D60A8AE096E00E94D60A8091B8
:1011D0000A06853609F1863670F4873471F1883451
:1011E00020F4853409F05AC014C08035D1F184361A
:1011F00009F054C03FC0883691F0893620F4873614
:1012000009F04CC024C0803779F1833709F046C01B
:101210002EC00E94770442C00E9472043FC08BEB34
:1012200092E00E94D60A81E08093560680910B06D8
:10123000803381F5109256062AC010928E04E4EC99
:10124000F7E0119287E0EC3CF807D9F727C010923D
:101250008E04EBE4F6E0119286E0E635F807D9F764
:101260001DC00E94B2071AC00E94540717C00E94F6
:10127000270814C080ED92E00E94D60A81E0809396
:10128000C20580910B06803329F41092C20587ECC9
:1012900092E002C08CEC92E00E94D60A8DED92E0C2
:1012A0000E94D60AEAE0F6E0119286E0EA32F807F8
:1012B000D9F708951DB88091F80580FF02C06D9A96
:1012C00001C06D988DB18091E50580FF02C06B9AD9
:1012D00001C06B988DB18091F60580FF02C06A9ABB
:1012E00001C06A988DB18091F705833091F0843008
:1012F00028F4813051F0823050F410C0853089F0EC
:10130000853048F0863051F407C0699A0AC0699A5E
:1013100003C0689A06C0689A709A04C08DB1836051
:101320008DB970988DB180658DB908951092F705CB
:101330001092F8051092E5051092F6050E945A09E0
:101340000895873008F086E08093F7050E945A09D7
:101350000895811181E08093F8050E945A0908954B
:10136000811181E08093E5050E945A090895811159
:1013700081E08093F6050E945A0908956C9B6C9A4F
:101380008FB9779BFECF8FB10895AF92BF92CF9266
:10139000DF92EF92FF920F931F93CF93DF93C82EAC
:1013A000D62EEE24FF24862F90E02AE9A22E25E0F7
:1013B000B22EA80EB91EEC01CB51DD4F01E010E0BA
:1013C0007BC0F50180818823C1F0DD2059F428B36A
:1013D0008881A80102C0440F551F8A95E2F7242B8B
:1013E00028BB26C022B38881F80102C0EE0FFF1F80
:1013F0008A95E2F72E2B22BB1BC0DD2069F428B3AF
:101400008881A80102C0440F551F8A95E2F7CA01DE
:101410008095822388BB0CC022B38881F80102C06A
:10142000EE0FFF1F8A95E2F7CF018095822382BBE2
:10143000F701EA51FA4F80810E94BE09F701E75097
:10144000FA4F8083F50180818823E1F0DD2069F483
:1014500028B38881A80102C0440F551F8A95E2F77E
:10146000CA018095822388BB24C022B38881F801F9
:1014700002C0EE0FFF1F8A95E2F7CF01809582230D
:1014800082BB17C0DD2059F428B38881A80102C0AF
:10149000440F551F8A95E2F7242B28BB0AC022B3BC
:1014A0008881F80102C0EE0FFF1F8A95E2F72E2B0C
:1014B00022BB0894E11CF11CEC1408F482CFDF91EC
:1014C000CF911F910F91FF90EF90DF90CF90BF9041
:1014D000AF900895FF920F931F93CF93DF93F82E51
:1014E000042F442379F488B39091E50221E030E0A1
:1014F00002C0220F331F9A95E2F7822788BBEB01C7
:1015000010E014C022B3E42FF0E0EB51FD4F308126
:1015100081E090E002C0880F991F3A95E2F72827F2
:1015200022BBEDCF89910E94BE091F5F1F15D0F32A
:10153000002369F488B39091E50221E030E002C015
:10154000220F331F9A95E2F7822788BB0FC022B380
:10155000E02FF0E0EB51FD4F308181E090E002C0E0
:10156000880F991F3A95E2F7282722BBDF91CF9188
:101570001F910F91FF90089510BC83E389B91BB8A8
:101580001AB8549A8898579A539A899A86E880BDCF
:1015900008955D9BFECF8CB908955D9BFECF8DE0D5
:1015A0008CB95D9BFECF8AE08CB90895FC0104C024
:1015B0005D9BFECF31968CB980818823C9F7089551
:1015C000FC0104C05D9BFECF31968CB980818823DD
:1015D000C9F70895FC0104C05D9BFECF31968CB91C
:1015E00080818823C9F75D9BFECF8DE08CB95D9B20
:1015F000FECF8AE08CB908950E94D60A5D9BFECF8B
:101600008DE08CB95D9BFECF8AE08CB908951F9266
:101610000F920FB60F9211248F939F93EF93FF9326
:101620009CB19093A10580919E058823A9F59D30DA
:1016300089F480919F05E82FF0E0E65FF94F108272
:101640008093090610929F051092A00581E0809377
:101650009E0522C08091A0058823F1F49F3511F0EA
:101660009B3321F481E08093A00516C0983031F4BB
:1016700080919F05882381F081500CC0903260F0EA
:1016800080919F058F3140F4E82FF0E0E65FF94F3D
:1016900090838F5F80939F05FF91EF919F918F9132
:1016A0000F900FBE0F901F9018950E944B0C0E9438
:1016B000D60A08950E94E40B0E94D60A08950E945B
:1016C000420D0E94D60A08950E945F0E0E94D60A1B
:1016D00008950E94BE0B0E94D60A08950E947B0FB7
:1016E0000E94D60A08950E94DE0F0E94D60A08952D
:1016F0000E94A20B0E94D60A08950E948C0B0E94A1
:10170000D60A08950E943A100E94D60A08950E94AF
:1017100078100E94D60A0895982F92959F70A9EE8E
:10172000B2E0FD01E90FF11D908190932A068F70C0
:10173000A80FB11D8C9180932B0610922C068AE283
:1017400096E00895EAE2F6E027E0482F50E060E3F3
:1017500031E3CA01022E02C0959587950A94E2F7FB
:10176000DF01119680FF02C0308301C06083FD015C
:10177000215078F71C928AE296E00895292F22954D
:101780002F70A9EEB2E0FD01E20FF11D2081209340
:101790002A069F70FD01E90FF11D908190932B06A1
:1017A000982F92959F70FD01E90FF11D9081909304
:1017B0002C068F70A80FB11D8C9180932D0610926E
:1017C0002E068AE296E00895292F22952F70A9EE21
:1017D000B2E0FD01E20FF11D208120932A069F70E7
:1017E000FD01E90FF11D908190932B06982F9295A2
:1017F0009F70FD01E90FF11D908190932C068F7071
:10180000FD01E80FF11D808180932D06872F8295C1
:101810008F70FD01E80FF11D808180932E067F708F
:10182000FD01E70FF11D808180932F06862F8295A1
:101830008F70FD01E80FF11D8081809330066F707D
:10184000A60FB11D8C9180933106109232068AE268
:1018500096E00895CF93DF93EC01FC010190002006
:10186000E9F73197E81BAAE3B6E080E202C08D9366
:101870006150E617E0F3CD018E0F911DFC0102C00F
:1018800089918D93AE17BF07D9F71C928AE396E032
:10189000DF91CF9108952F923F924F925F926F9276
:1018A0007F928F929F92AF92BF92CF92DF92EF92F0
:1018B000FF920F931F93DF93CF930F92CDB7DEB7B5
:1018C0003B014C012983242E85E0841710F435E078
:1018D000232EC401B30120E030E040E050E00E943C
:1018E0008A1687FD05C02AE2422E26E0522E0BC042
:1018F0008DE280932A0697FA909497F890949BE251
:10190000492E96E0592EC401B3010E94DE125B01FC
:101910006C01611571058105910521F480E3D20107
:101920008D932D0186017501332423C0C801B701B1
:101930002AE030E040E050E00E940D1AE32DF0E094
:10194000EE55FA4F6083E61AF10801091109E11416
:10195000F1040105110561F0C801B7012AE030E08A
:1019600040E050E00E940D1AC901DA017C018D01AE
:101970003394E114F10401051105C1F6C601B50166
:101980000E946C179B01AC01C401B3010E94561464
:101990007B018C018AEAA82E85E0B82E6501822C95
:1019A00099243501680C791C22C0C801B70120E0D8
:1019B00030E040E251E40E94B4147B018C010E94AB
:1019C000DE12F6016083662379F070E0882777FDE8
:1019D0008095982F0E94BA169B01AC01C801B701EF
:1019E0000E9456147B018C010894C11CD11CC614A2
:1019F000D704D9F6932D9150A92FBB27A7FDB095F9
:101A0000AE55BA4F07C08C91805DF20180832901E9
:101A10009150119792012F5F3F4F97FFF4CF8EE2C5
:101A2000D2018C93F20105C0D5018D915D01805DDD
:101A300080833196AC14BD04B9F7280D391DF90126
:101A40001082F981FF2319F42AE236E006C08AE207
:101A500096E069810E942A0C9C01C9010F90CF91E8
:101A6000DF911F910F91FF90EF90DF90CF90BF908B
:101A7000AF909F908F907F906F905F904F903F902E
:101A80002F900895BF92CF92DF92EF92FF920F9323
:101A90001F93CF93DF938B019C01B42E97FF0DC052
:101AA0008DE280932A06CC24DD247601C01AD10A67
:101AB000E20AF30ACBE2D6E004C06B017C01CAE281
:101AC000D6E080E0C8168AECD8068AE9E8068BE3FF
:101AD000F80658F0C701B60120E03AEC4AE95BE3AA
:101AE0000E940D1A205D299309C080E0C81681EE7E
:101AF000D80685EFE80685E0F80688F0C701B6014C
:101B000020E03AEC4AE95BE30E940D1A20E031EE56
:101B100045EF55E00E940D1A205D299309C080E829
:101B2000C81686E9D80688E9E80680E0F80688F055
:101B3000C701B60120E031EE45EF55E00E940D1AD5
:101B400020E836E948E950E00E940D1A205D29930B
:101B500009C080E4C81682E4D8068FE0E80680E079
:101B6000F80688F0C701B60120E836E948E950E0F8
:101B70000E940D1A20E432E44FE050E00E940D1A5A
:101B8000205D299309C080EAC81686E8D80681E05E
:101B9000E80680E0F80688F0C701B60120E432E4E8
:101BA0004FE050E00E940D1A20EA36E841E050E094
:101BB0000E940D1A205D299309C080E1C81687E2B2
:101BC000D80680E0E80680E0F80688F0C701B60194
:101BD00020EA36E841E050E00E940D1A20E137E2A9
:101BE00040E050E00E940D1A205D299309C088EE64
:101BF000C81683E0D80680E0E80680E0F80688F0A2
:101C0000C701B60120E137E240E050E00E940D1A22
:101C100028EE33E040E050E00E940D1A205D299349
:101C200006C084E6C816D104E104F10488F0C701B7
:101C3000B60128EE33E040E050E00E940D1A24E6A1
:101C400030E040E050E00E940D1A205D299306C06C
:101C50008AE0C816D104E104F10480F0C701B6019E
:101C600024E630E040E050E00E940D1A2AE030E027
:101C700040E050E00E940D1A205D2993C701B60193
:101C80002AE030E040E050E00E940D1A605D688379
:101C90001982BB2019F42AE236E006C08AE296E0F7
:101CA0006B2D0E942A0C9C01C901DF91CF911F91DD
:101CB0000F91FF90EF90DF90CF90BF900895DF924B
:101CC000EF92FF920F931F93CF93DF937B018C01D1
:101CD000D42E80E0E8168AECF8068AE908078BE340
:101CE000180770F0C801B70120E03AEC4AE95BE35D
:101CF0000E940D1A205D20932A06CBE2D6E00BC08D
:101D000080E0E81681EEF80685EF080785E0180701
:101D100098F0CAE2D6E0C801B70120E03AEC4AE9FF
:101D20005BE30E940D1A20E031EE45EF55E00E9482
:101D30000D1A205D29930BC080E8E81686E9F806A5
:101D400088E9080780E0180798F0CAE2D6E0C801E1
:101D5000B70120E031EE45EF55E00E940D1A20E872
:101D600036E948E950E00E940D1A205D29930BC026
:101D700080E4E81682E4F8068FE0080780E01807A0
:101D800098F0CAE2D6E0C801B70120E836E948E990
:101D900050E00E940D1A20E432E44FE050E00E942F
:101DA0000D1A205D29930BC080EAE81686E8F80634
:101DB00081E0080780E0180798F0CAE2D6E0C80181
:101DC000B70120E432E44FE050E00E940D1A20EA0F
:101DD00036E841E050E00E940D1A205D29930BC0C7
:101DE00080E1E81687E2F80680E0080780E018073F
:101DF00098F0CAE2D6E0C801B70120EA36E841E02F
:101E000050E00E940D1A20E137E240E050E00E94CD
:101E10000D1A205D29930BC088EEE81683E0F806C2
:101E200080E0080780E0180798F0CAE2D6E0C80111
:101E3000B70120E137E240E050E00E940D1A28EEA1
:101E400033E040E050E00E940D1A205D299308C065
:101E500084E6E816F1040105110598F0CAE2D6E01F
:101E6000C801B70128EE33E040E050E00E940D1AAF
:101E700024E630E040E050E00E940D1A205D2993F6
:101E80000BC08AE0E816F1040105110518F4CAE256
:101E9000D6E012C0CAE2D6E0C801B70124E630E0BD
:101EA00040E050E00E940D1A2AE030E040E050E0AF
:101EB0000E940D1A205D2993C801B7012AE030E085
:101EC00040E050E00E940D1A605D68831982DD20B9
:101ED00019F42AE236E006C08AE296E06D2D0E94EF
:101EE0002A0C9C01C901DF91CF911F910F91FF90A6
:101EF000EF90DF900895CF93DF939C01462F97FFDB
:101F00000AC08DE280932A06EE27FF27E21BF30B1F
:101F1000CBE2D6E003C0FC01CAE2D6E087E2E031C2
:101F2000F80740F0CF0160E177E20E94E619605DBA
:101F3000699304C083E0E83EF80760F0CF0160E1F8
:101F400077E20E94E61968EE73E00E94E619605D90
:101F5000699303C0E436F10560F0CF0168EE73E0E9
:101F60000E94E61964E670E00E94E619605D6993DC
:101F700003C0EA30F10558F0CF0164E670E00E943A
:101F8000E6196AE070E00E94E619605D6993CF018E
:101F90006AE070E00E94E619805D8883198244231C
:101FA00019F42AE236E006C08AE296E0642F0E9425
:101FB0002A0C9C01C901DF91CF9108959C01462F05
:101FC00087E22031380758F0C90160E177E20E94CA
:101FD000E619605D60932A06EBE2F6E006C083E056
:101FE000283E380770F0EAE2F6E0C90160E177E2E6
:101FF0000E94E61968EE73E00E94E619605D619345
:1020000005C02436310570F0EAE2F6E0C90168EE59
:1020100073E00E94E61964E670E00E94E619605DD4
:10202000619308C02A30310518F4EAE2F6E00DC0E9
:10203000EAE2F6E0C90164E670E00E94E6196AE0AF
:1020400070E00E94E619605D6193C9016AE070E08A
:102050000E94E619805D80831182442319F42AE2EC
:1020600036E006C08AE296E0642F0E942A0C9C01AA
:10207000C9010895982F362F87FF08C08DE28093FD
:102080002A06292F2195EBE2F6E003C0282FEAE289
:10209000F6E0243668F0822F90E068EE73E00E944C
:1020A000FA1964E670E00E94FA19605D619302C05B
:1020B0002A3050F0822F64E60E94DA19892F6AE0F4
:1020C0000E94DA19805D8193822F6AE00E94DA19FA
:1020D000905D90831182332319F42AE236E006C022
:1020E0008AE296E0632F0E942A0C9C01C9010895A0
:1020F0001F93482F162F843678F090E068EE73E037
:102100000E94FA1964E670E00E94FA19605D60931B
:102110002A062BE236E007C08A3018F4EAE2F6E03D
:102120000DC02AE236E0842F64E60E94DA19892F76
:102130006AE00E94DA19805DF9018193842F6AE0D8
:102140000E94DA19905D90831182112319F42AE21A
:1021500036E006C08AE296E0612F0E942A0C9C01BC
:10216000C9011F9108951F920F920FB60F9211246B
:102170008F939F93AF93BF938091B3059091B405D4
:10218000A091B505B091B6050196A11DB11D809332
:10219000B3059093B405A093B505B093B605BF9170
:1021A000AF919F918F910F900FBE0F901F90189538
:1021B000CF92DF92EF92FF921F93CF93DF930E9413
:1021C000C7030E94BC0A0E94960988E085BD85B5B8
:1021D000836085BD8CE783BD89B7806889BF7894AB
:1021E0008AEF92E00E94D60A6091B3057091B4051F
:1021F0008091B5059091B60520E137E240E050E0CE
:102200000E940D1A6115710581059105D9F482E2CC
:1022100093E00E94D60A6091B3057091B405809155
:10222000B5059091B60528EE33E040E050E00E94FD
:102230000D1ACA01B90146E00E94640B89E293E0DD
:102240000E94D60AC29884EF91E028EC30E0F901B0
:102250003197F1F70197D9F7C29A80E197E2019798
:10226000F1F78FE293E00E94D60A6091B305709176
:10227000B4058091B5059091B6054AE00E94640BC3
:1022800085E493E00E94D60A0E9449028AE493E022
:102290000E94D60A6091B3057091B4058091B5058E
:1022A0009091B6054AE00E94640B85E493E00E9499
:1022B000D60A82E693E00E94D60AC8ECD0E012C0AB
:1022C00083E893E00E94D60A0E94B3000E947D0B2F
:1022D0008AE00E94C90A82E09DE0FE013197F1F791
:1022E0000197D9F70E94B800882351F385E993E05C
:1022F0000E94D60A6091B3057091B4058091B5052E
:102300009091B60528EE33E040E050E00E940D1AAF
:10231000CA01B90146E00E94640B89E293E00E9481
:10232000D60A86EB93E00E94D60A20E23EE403C080
:10233000C9010197F1F780919E058823C9F3109296
:102340009E0583EF93E00E94D60AC8ECD0E05BC004
:102350000E94A1000E94690B89E00E94C90A8CE7D3
:102360000E94C90A0E948F000E94690B89E00E94A6
:10237000C90A8CE70E94C90A0E947D000E94690B6D
:1023800089E00E94C90A8CE70E94C90A0E946B007A
:102390000E94690B89E00E94C90A8CE70E94C90A61
:1023A0000E9459000E94690B89E00E94C90A8CE7CB
:1023B0000E94C90A86E294E00E9449000E947D0BB7
:1023C00089E00E94C90A8CE70E94C90A87E294E06A
:1023D0000E9449000E947D0B89E00E94C90A8CE797
:1023E0000E94C90A8AE00E94C90A80EA9FE0FE01B1
:1023F0003197F1F70197D9F780EA9FE0FE01319715
:10240000F1F70197D9F780919E05882309F4A0CFB1
:1024100010929E0588ECC82ED12C89C00E946B00BA
:102420007C010E94A1000E94690B89E00E94C90AF8
:102430008CE70E94C90A0E948F000E94690B89E004
:102440000E94C90A8CE70E94C90A0E947D000E946E
:10245000690B89E00E94C90A8CE70E94C90A0E94A0
:102460006B000E94690B89E00E94C90A8CE70E94F8
:10247000C90A0E9459000E94690B89E00E94C90A9A
:102480008CE70E94C90A0E946B00892B89F18BE3BB
:1024900094E00E94D60A0E946B0066E00E94730BD3
:1024A00085E494E00E94D60A20C080E161E00E94A9
:1024B000E300182F81E20E94C90A812F64E00E9484
:1024C000870B8AE00E94C90AC0E0D0E00AC0FE0182
:1024D000ED53FA4F80810E947D0B80E20E94C90A71
:1024E0002196C117A0F3E11AF108E114F104E9F60D
:1024F0008AE00E94C90A80EA9FE0F6013197F1F76D
:102500000197D9F780EA9FE0F6013197F1F701973B
:10251000D9F780EA9FE0F6013197F1F70197D9F7F3
:1025200080EA9FE0F6013197F1F70197D9F78091A2
:102530009E05882309F472CF10929E05C8ECD0E066
:1025400084E594E00E94D60A07C088EE93E0FE017D
:102550003197F1F70197D9F780919E058823A9F368
:1025600010929E0580910A06883521F480910B0611
:10257000883529F09091090620E030E00FC0809165
:102580000C068835B9F710C0F901E65FF94F808174
:10259000F901ED52FA4F80832F5F3F4F2917A0F3C7
:1025A000892F0E94C701CCCF80E090E0DF91CF91CE
:1025B0001F91FF90EF90DF90CF900895EF92FF92E0
:1025C0000F931F937B018C0120E030E040E05FE43B
:1025D0000E945A1688238CF0C801B70120E030E031
:1025E00040E05FE40E9456140E9418179B01AC0162
:1025F000205030404040504806C0C801B7010E94FA
:1026000018179B01AC01B901CA011F910F91FF90EE
:10261000EF900895A0E0B0E0E0E1F3E10C942F1A10
:10262000DC012B01FA019C91923008F439C1EB01D5
:102630008881823008F433C1943069F4843009F021
:102640002FC111969C9111978981981709F428C17F
:10265000AFE8B4E025C1843009F421C18230A9F487
:10266000923009F01DC19A01AD0188E0EA0109909C
:10267000AE01E90109929E018150C1F7E201898111
:1026800011969C918923818308C1923009F407C176
:1026900012962D903C901397EB018A819B811496A2
:1026A000AD90BD90CD90DC901797EC80FD800E81B1
:1026B0001F819101281B390BB90137FF04C0662720
:1026C0007727621B730B603271050CF061C0121624
:1026D00013066CF537014801062E04C096948794C2
:1026E000779467940A94D2F721E030E040E050E01C
:1026F00004C0220F331F441F551F6A95D2F7215083
:102700003040404050402E213F214023512321158D
:1027100031054105510521F021E030E040E050E075
:1027200079018A01E628F728082919293CC0232BBA
:10273000D1F1260E371E35014601062E04C09694AF
:102740008794779467940A94D2F721E030E040E0D0
:1027500050E004C0220F331F441F551F6A95D2F763
:1027600021503040404050402A213B214C215D21E6
:10277000211531054105510521F021E030E040E00F
:1027800050E059016A01A628B728C828D9280BC0EB
:10279000821593052CF01C01AA24BB24650103C0FB
:1027A000EE24FF24870111969C91D20111968C9101
:1027B000981709F445C0992339F0A80197012A19FF
:1027C0003B094C095D0906C0A60195012E193F0978
:1027D000400B510B57FD08C01182338222822483A3
:1027E0003583468357831DC081E0818333822282F3
:1027F00088279927DC01821B930BA40BB50B8483DC
:102800009583A683B7830DC0220F331F441F551F26
:1028100024833583468357838281938101979383F1
:1028200082832481358146815781DA01C90101976C
:10283000A109B1098F5F9F4FAF4FBF4328F30BC072
:10284000918333822282EA0CFB1C0C1D1D1DE48245
:10285000F5820683178383E0808324813581468156
:10286000578157FF1AC0C901AA2797FDA095BA2F13
:1028700081709070A070B0705695479537952795E8
:10288000822B932BA42BB52B84839583A683B783AC
:1028900082819381019693838283DF0101C0D201FB
:1028A000CD01CDB7DEB7E2E10C944B1AA0E2B0E067
:1028B000ECE5F4E10C943B1A69837A838B839C8367
:1028C0002D833E834F835887E9E0EE2EF12CEC0EEA
:1028D000FD1ECE010196B7010E9409198E010F5EFF
:1028E0001F4FCE010596B8010E9409198A8991E00F
:1028F00089278A8BC701B801AE01475E5F4F0E94EE
:102900000A130E943418A096E6E00C94571AA0E22D
:10291000B0E0EDE8F4E10C943B1A69837A838B8391
:102920009C832D833E834F835887F9E0EF2EF12C53
:10293000EC0EFD1ECE010196B7010E9409198E0111
:102940000F5E1F4FCE010596B8010E940919C701FD
:10295000B801AE01475E5F4F0E940A130E9434180F
:10296000A096E6E00C94571AA0E2B0E0EAEBF4E19E
:102970000C942F1A69837A838B839C832D833E83E7
:102980004F835887CE010196BE01675F7F4F0E943B
:102990000919CE010596BE016F5E7F4F0E9409198D
:1029A0009985923088F089898230C8F0943019F482
:1029B000823051F404C0843029F4923081F48FE8DD
:1029C00094E0C6C0923049F420E09A858A89981331
:1029D00021E02A87CE010996BBC0823049F420E06D
:1029E0009A858A89981321E02A8BCE014196B0C03E
:1029F0002D843E844F8458886D887E888F88988C7B
:102A0000EE24FF248701AA24BB24650140E050E0A6
:102A100060E070E0E0E0F0E0C10181709070892B2F
:102A2000E9F0E60CF71C081D191D9A01AB012A0DEF
:102A30003B1D4C1D5D1D80E090E0A0E0B0E0E61481
:102A4000F7040805190520F481E090E0A0E0B0E06B
:102A5000BA01A901480F591F6A1F7B1FAA0CBB1C92
:102A6000CC1CDD1C97FE08C081E090E0A0E0B0E047
:102A7000A82AB92ACA2ADB2A3196E032F10549F0A0
:102A8000660C771C881C991C56944794379427949D
:102A9000C3CFFA85EA892B893C898B859C85280FD1
:102AA000391F2E5F3F4F17C0CA0181709070892B6C
:102AB00061F016950795F794E79480E090E0A0E028
:102AC000B0E8E82AF92A0A2B1B2B769567955795CB
:102AD00047952F5F3F4F77FDE7CF0CC0440F551F41
:102AE000661F771F17FD4160EE0CFF1C001F111FB2
:102AF00021503040403090E0590790E0690790E461
:102B0000790760F32B8F3C8FDB01CA018F779070C0
:102B1000A070B07080349105A105B10561F447FD46
:102B20000AC0E114F1040105110529F0405C5F4F72
:102B30006F4F7F4F40781A8EFE1711F081E08A8F19
:102B40004D8F5E8F6F8F78A383E0898FCE0149967A
:102B50000E943418A096E2E10C944B1AA8E1B0E070
:102B6000E4EBF5E10C94371A69837A838B839C83B9
:102B70002D833E834F835887B9E0EB2EF12CEC0E6A
:102B8000FD1ECE010196B7010E9409198E010F5E4C
:102B90001F4FCE010596B8010E94091929852230E0
:102BA00008F47EC03989323010F4B8017CC08A85BF
:102BB0009A8989278A87243011F0223031F423172B
:102BC00009F06EC06FE874E06EC0343039F41D86D1
:102BD0001E861F86188A1C861B8604C0323021F48C
:102BE00084E08987B7015FC02B853C858B899C89F0
:102BF000281B390B3C872B87ED84FE840F851889B1
:102C0000AD88BE88CF88D88CEA14FB040C051D055E
:102C100040F4EE0CFF1C001F111F215030403C8778
:102C20002B8720E030E040E050E080E090E0A0E042
:102C3000B0E460E070E0EA14FB040C051D0540F010
:102C4000282B392B4A2B5B2BEA18FB080C091D0992
:102C5000B695A79597958795EE0CFF1C001F111F41
:102C60006F5F7F4F6F31710531F7DA01C9018F77DF
:102C70009070A070B07080349105A105B10561F429
:102C800027FD0AC0E114F1040105110529F0205CBB
:102C90003F4F4F4F5F4F20782D873E874F87588B90
:102CA000BE01675F7F4FCB010E9434186896EAE04F
:102CB0000C94531AA8E1B0E0E0E6F6E10C943B1A5C
:102CC00069837A838B839C832D833E834F835887CC
:102CD00089E0E82EF12CEC0EFD1ECE010196B70125
:102CE0000E9409198E010F5E1F4FCE010596B80193
:102CF0000E9409198985823040F08989823028F044
:102D0000C701B8010E94811901C08FEF6896E6E003
:102D10000C94571AA8E1B0E0E0E9F6E10C943B1AF4
:102D200069837A838B839C832D833E834F8358876B
:102D300089E0E82EF12CEC0EFD1ECE010196B701C4
:102D40000E9409198E010F5E1F4FCE010596B80132
:102D50000E9409198985823040F08989823028F0E3
:102D6000C701B8010E94811901C081E06896E6E0C0
:102D70000C94571AA8E0B0E0E0ECF6E10C94381A95
:102D80009B01AC0183E08983DA01C9018827B7FD83
:102D900083959927AA27BB27B82E21153105410510
:102DA000510519F482E089833AC08823A9F02030C4
:102DB00080E0380780E0480780E8580729F460E0A1
:102DC00070E080E09FEC30C0EE24FF248701E21A1F
:102DD000F30A040B150B02C079018A018EE1C82E9B
:102DE000D12CDC82CB82ED82FE820F831887C80152
:102DF000B7010E94E51701971816190684F4082EEA
:102E000004C0EE0CFF1C001F111F0A94D2F7ED82C4
:102E1000FE820F831887C81AD90ADC82CB82BA8255
:102E2000CE0101960E9434182896E9E00C94541AB9
:102E3000ACE0B0E0EEE1F7E10C943F1A69837A83ED
:102E40008B839C83CE010196BE016B5F7F4F0E94F6
:102E500009198D81823061F1823050F1843021F482
:102E60008E81882351F12EC02F81388537FD20C0F7
:102E70006E812F3131051CF06623F9F023C08EE1FD
:102E800090E0821B930B29853A854B855C8504C0B5
:102E900056954795379527958A95D2F76623B1F0D1
:102EA00050954095309521953F4F4F4F5F4F0EC045
:102EB00020E030E040E050E009C02FEF3FEF4FEF5F
:102EC0005FE704C020E030E040E050E8B901CA010B
:102ED0002C96E2E00C945B1AA8E0B0E0E2E7F7E1A0
:102EE0000C94371A7B018C016115710581059105E0
:102EF00019F482E0898360C083E089838EE1C82E63
:102F0000D12CDC82CB82ED82FE820F831887C80130
:102F1000B7010E94E517FC013197F7FF3BC022275C
:102F200033272E1B3F0B57016801022E04C0D69495
:102F3000C794B794A7940A94D2F740E050E060E0B9
:102F400070E081E090E0A0E0B0E004C0880F991F3D
:102F5000AA1FBB1F2A95D2F70197A109B1098E219B
:102F60009F21A023B1230097A105B10521F041E0E5
:102F700050E060E070E04A295B296C297D294D838F
:102F80005E836F8378878EE190E08E1B9F0B9C831E
:102F90008B8312C0309781F00E2E04C0EE0CFF1C04
:102FA000001F111F0A94D2F7ED82FE820F8318874B
:102FB000CE1ADF0ADC82CB821A82CE0101960E94F1
:102FC00034182896EAE00C94531AEF92FF920F936C
:102FD0001F937B018C0180E0E81680E0F80681E019
:102FE000080780E0180788F48FEFE816F104010560
:102FF000110531F028F088E090E0A0E0B0E017C0C3
:1030000080E090E0A0E0B0E012C080E0E81680E050
:10301000F80680E0080781E0180728F088E190E0D2
:10302000A0E0B0E004C080E190E0A0E0B0E020E2E9
:1030300030E040E050E0281B390B4A0B5B0B04C02A
:1030400016950795F794E7948A95D2F7F701E95614
:10305000FB4F8081281B310941095109C9011F918A
:103060000F91FF90EF900895DF92EF92FF920F93F0
:103070001F93FC01E480F58006811781D180808157
:10308000823048F480E090E0A0E1B0E0E82AF92A3C
:103090000A2B1B2BA5C0843009F49FC0823021F479
:1030A000EE24FF24870105C0E114F1040105110598
:1030B00019F4E0E0F0E096C0628173819FEF62381E
:1030C00079070CF05BC022E83FEF261B370B2A3153
:1030D00031052CF020E030E040E050E02AC0B8019B
:1030E000A701022E04C076956795579547950A94D7
:1030F000D2F781E090E0A0E0B0E004C0880F991F13
:10310000AA1FBB1F2A95D2F70197A109B1098E21E9
:103110009F21A023B1230097A105B10521F081E0F3
:1031200090E0A0E0B0E09A01AB01282B392B4A2BAC
:103130005B2BDA01C9018F779070A070B07080347A
:103140009105A105B10539F427FF09C0205C3F4F67
:103150004F4F5F4F04C0215C3F4F4F4F5F4FE0E048
:10316000F0E02030A0E03A07A0E04A07A0E45A07C8
:1031700010F0E1E0F0E079018A0127C060387105C4
:1031800064F5FB01E158FF4FD801C7018F779070BC
:10319000A070B07080349105A105B10539F4E7FE47
:1031A0000DC080E490E0A0E0B0E004C08FE390E0C8
:1031B000A0E0B0E0E80EF91E0A1F1B1F17FF05C0B4
:1031C00016950795F794E794319687E0169507953D
:1031D000F794E7948A95D1F705C0EE24FF24870180
:1031E000EFEFF0E06E2F679566276795902F9F773A
:1031F000D794DD24D7948E2F8695492F462B582FB0
:103200005D29B701CA011F910F91FF90EF90DF90E8
:103210000895FC01DB01408151812281622F6F778B
:1032200070E0221F2227221F9381892F880F822B73
:10323000282F30E0991F9927991F11969C93119779
:1032400021153105A9F5411551056105710511F4E7
:1032500082E037C082E89FEF13969C938E9312977B
:103260009A01AB0167E0220F331F441F551F6A9577
:10327000D1F783E08C930DC0220F331F441F551FDD
:1032800012968D919C911397019713969C938E9310
:103290001297203080E0380780E0480780E4580724
:1032A00058F314962D933D934D935C93179708957F
:1032B0002F3F310579F4411551056105710519F468
:1032C00084E08C93089564FF03C081E08C9312C066
:1032D0001C9210C02F57304013963C932E93129798
:1032E00083E08C9387E0440F551F661F771F8A95F4
:1032F000D1F7706414964D935D936D937C931797FB
:1033000008951F93DC01FB019C91923008F447C0A3
:103310008081823008F443C0943051F411961C919E
:10332000843099F58181682F70E0611B71093FC07D
:10333000843021F0923031F48230B9F181818823D8
:1033400089F12DC011961C9111978230F1F0818185
:103350001817D9F412962D913C911397828193817D
:103360008217930794F028173907BCF014968D91B3
:103370009D910D90BC91A02D24813581468157816E
:10338000281739074A075B0718F4112341F00AC0D0
:1033900082179307A407B50740F4112319F061E0E1
:1033A00070E005C06FEF7FEF02C060E070E0CB011E
:1033B0001F910895991B79E004C0991F961708F092
:1033C000961B881F7A95C9F780950895AA1BBB1B89
:1033D00051E107C0AA1FBB1FA617B70710F0A61B15
:1033E000B70B881F991F5A95A9F780959095BC0136
:1033F000CD01089597FB092E07260AD077FD04D04A
:10340000E5DF06D000201AF4709561957F4F08958E
:10341000F6F7909581959F4F0895A1E21A2EAA1B69
:10342000BB1BFD010DC0AA1FBB1FEE1FFF1FA21774
:10343000B307E407F50720F0A21BB30BE40BF50B71
:10344000661F771F881F991F1A9469F760957095FA
:10345000809590959B01AC01BD01CF0108952F92FD
:103460003F924F925F926F927F928F929F92AF9214
:10347000BF92CF92DF92EF92FF920F931F93CF9361
:10348000DF93CDB7DEB7CA1BDB0B0FB6F894DEBFF8
:103490000FBECDBF09942A88398848885F846E841E
:1034A0007D848C849B84AA84B984C884DF80EE8068
:1034B000FD800C811B81AA81B981CE0FD11D0FB671
:1034C000F894DEBF0FBECDBFED010895F894FFCF95
:1034D0006C6173745F726561645F706F696E74654F
:1034E000723A000A6F66667365743A000A73746113
:1034F00072745F616464726573733A0049737375C3
:10350000696E6720536F636B6574206F70656E2002
:10351000636F6D6D616E642E204E4F570A00536FBE
:10352000636B6574203020737461747573206973E4
:103530003A0049737375696E6720536F636B6574E6
:10354000204C495354454E20636F6D6D616E642E5F
:10355000204E4F570A0073657474696E67206F665A
:103560002041546D65676120696E7465726E616C8F
:103570002041444320656E61626C65207265676915
:103580007374657273206973206E6F742073757025
:10359000706F727465642E207965742E0A000A209B
:1035A00073657420656E61626C6520626974732056
:1035B0006F662041443737313920506F72742000D4
:1035C00020746F200020746F20307846460A002057
:1035D000746F20307830300A000A20736F6D657484
:1035E00068696E672077726F6E670A007573617223
:1035F000745F72785F6275666665725F696E646536
:10360000783A20000A2075736172745F72785F6285
:1036100075666665725B325D3A20000A20757361DB
:1036200072745F72785F6275666665725B345D3A6C
:10363000200020207C0020204F6F5220207C000A98
:10364000207072696E74696E6720766F6C74616742
:10365000657320696E206D563A0A002020200052C2
:103660003A000A207072696E74696E67206D656138
:10367000737572656420726573697374616E6365D6
:1036800020696E206B6F686D733A0A00200020205D
:103690002020202020202000616463207374617446
:1036A00075733A0A00616437373139207374617475
:1036B00075733A0A0074696D653A00207365632E6C
:1036C0000A00616463206D656173757265642061D1
:1036D0006C6C3A200020747275650A0066616C7328
:1036E000650A00616437373139206D656173757221
:1036F000656420616C6C3A200061646320637572BC
:1037000072656E74206368616E6E656C3A00616408
:10371000373731392063757272656E742063686162
:103720006E6E656C3A00676F743A000A6865617284
:10373000746265617420006F66660A006F6E0A002D
:103740000A6465627567206D6F646520000A7265A2
:103750006164793F00040304053031323334353677
:1037600037383941424344454600537461727420EE
:103770006F662074657374206669726D7761726517
:10378000202830362E30352E313129206E6F773A91
:103790000A0074696D653A20007365632E0A00574C
:1037A0003533303020696E697420626567696E73E5
:1037B0002061743A006D732E0A0057353330302083
:1037C000696E69742066696E6973686564206174E6
:1037D0003A005761697420666F7220504320746FFD
:1037E00020636F6E6E65637420746F204653432EA2
:1037F0002E2E00536F636B65742073746174757340
:103800002069733A00636F6E6E656374696F6E2032
:10381000746F2050432065737461626C69736865CE
:10382000642061743A00526561647920746F206984
:103830006E7665737469676174652C20776861744E
:1038400027732068617070656E696E67206E657899
:10385000743F202D2048495420454E544552202D78
:10386000200A0053305F54585F465352097C53304E
:103870005F54585F5244097C53305F54585F57522D
:10388000097C53305F52585F525352097C53305F6A
:1038900052585F5244097C20307830343236207CD4
:1038A00020307830343237207C0A000A5265616457
:1038B000696E67200020622066726F6D2057353177
:1038C00030300A00456E7465722074686520737428
:1038D00072696E6720746F2073656E6420746F2048
:1038E0005043206F7220225858582220696E206F52
:1038F0007264657220746F20717569740A0001002A
:1039000000000000000000000102020303030304A2
:10391000040404040404040505050505050505055E
:10392000050505050505050606060606060606063E
:103930000606060606060606060606060606060627
:10394000060606060606060707070707070707070E
:1039500007070707070707070707070707070707F7
:1039600007070707070707070707070707070707E7
:1039700007070707070707070707070707070707D7
:1039800007070707070707080808080808080808BE
:1039900008080808080808080808080808080808A7
:1039A0000808080808080808080808080808080897
:1039B0000808080808080808080808080808080887
:1039C0000808080808080808080808080808080877
:1039D0000808080808080808080808080808080867
:1039E0000808080808080808080808080808080857
:1039F0000808080808080808080808080808080847
:083A0000080808080808080086
:00000001FF
